:020000040000FA
:1000000083161E308500F030860081138312EF3096
:100010009F0086000430A0009F0C1F08860031203E
:1000200006080F38A100A109031D1928A00B0C28F0
:10003000072883160030860083129F091F080F3996
:100040009F002108F0399F041F0886001130A1008D
:10005000A103210839201F02031D2828210886003A
:100060003028FA30A300A200A20B3428A30B3328B7
:100070000800820711341234143418342134223425
:100080002434283441344234443448348134823472
:100090008434883430343134323433343434353485
:1000A00036343734383438344134423443344434C9
:0400B0004534463459
:02400E00F13F80
:00000001FF
